:1000000013298030A100FE30A7200130A7207530D1
:10001000A7003030BF28A101A117AF00AF08031D12
:100020001328030114280130AF020310A20CA20C04
:10003000A20CC0302205403EAF07FE30A7202F089B
:10004000A728A101A117AF00FE30A7202F08A728DD
:10005000A401AA00AB01A01124080319A0150530C2
:10006000A3002730A900103041200330A900E83058
:100070004120A90164304120A9010A3041202A0809
:100080004828A8002B08A7002A08A600DD2026087B
:10009000A600A3030319A011240803195228230260
:1000A000031859282608031DA011A0195928303E0D
:1000B000A7280800AD0006118611831606118611C7
:1000C0000F30860583122D08A01884283E30A70023
:1000D0008030BF203330AC0098201330A700883028
:1000E000BF2098206430BE2098206430BE2022308B
:1000F000AC009820283083200C30832006308320E9
:10010000A0142D0884282014AC00201C92288611ED
:10011000033C031C972897200730A700D030BF204E
:10012000031408002014FE3C0319A5288615201C82
:10013000201006150F3086052C08F03986040611AC
:10014000AC0E201898283230BE202D080F29A11B94
:100150005A28080083178001840AFF3E031DAB283C
:100160000F29A901A800FF30A807031CA907031C39
:100170000F290330A700DF30BF20B328A701E83ED6
:10018000A600A709FC30031CC828A6070318C52829
:10019000A6070000A70FC5282618CE28A61CD2281F
:1001A0000000D2280800013EAD000A30A800A901D5
:1001B000DD20AD0BD8282A080800AB01AA011030B9
:1001C000AC00270DAA0DAB0D2808AA022908031CB4
:1001D000290FAB020318F3282808AA0729080318D7
:1001E000290FAB070310A60DA70DAC0BE1282608BD
:1001F0000F291030B000A701A601AD0CAC0C031CF8
:1002000007292808A60729080318290FA707A70CFC
:10021000A60CAB0CAA0CB00BFD282A080F298313DF
:10022000831203130800A00107309F00E0308316FB
:100230008500FF30860081138312850186012030FE
:1002400084006030AB20A03084005030AB202030E0
:1002500084003030AA20C830B120012077305A20E5
:100260005A205A202E305A2070305A2069305A2095
:1002700063305A2062305A208030A100C0302120E3
:1002800061305A2073305A2069305A2063305A2026
:100290002E305A206E305A206C305A200B30A90074
:1002A000B830B220012044305A2043305A20463022
:1002B0005A2031305A2036305A2055305A204B308F
:1002C0005A2045305A208030A100C23021205630BB
:1002D0005A202D305A2032305A200730A900D03011
:1002E000B220012041305A2064305A206A305A200E
:1002F00075305A2073305A2074305A2020305A20DA
:100300004C305A208030A100C030212044305A2087
:1003100052305A2086189229851F90290514912958
:1003200005108A29012053305A2065305A20613047
:100330005A2072305A2063305A2068305A202030B8
:100340005A2073305A208030A100C03021206930FB
:100350005A2067305A206E305A2061305A206C3053
:100360005A2049148316051283120512392AC20134
:100370003B03A500C80148082502031CCF29F22130
:10038000C91CCC294808A200A601A20A0314A60D84
:10039000A20BC7292608C204C80A031DBB294208AC
:1003A000B100B201B20CB10CB20CB10CB20CB10C78
:1003B000B20CB10C0F30B2053108AC003208AD0000
:1003C0000A30A800A901F920B1002B08B2004208A8
:1003D000B300B4010F30B3050030B4053108330762
:1003E000C2000800B801B9010618072A0130B1207F
:1003F000B80A0319B90A0B303902031C062A031D77
:10040000052AB9303802031C062A722CF4299B30C5
:10041000B1208310061883148318C914831CC910D3
:10042000491C262A4308B100B2010310B10DB20DD8
:10043000B10DB20DB10DB20D3108A6003208A70002
:100440003A30A800A901DD20BC002F2A0301491978
:10045000013EC918013A03194911031D4915C30A80
:1004600085140130A900F430B2208510F030B1209D
:100470000800BA01C3014912491AC82AB801B901D2
:10048000061C532AB80A0319B90A0130B120AF304B
:100490003902031C522A031D512AC9303802031C99
:1004A000522A722C402AB801B9010618852AB80AC6
:1004B0000319B90A0A30B1204918792A38080B3AC9
:1004C0003904031D642A782A3808193A3904031DAF
:1004D0006B2A8514782A38084B3A3904031D722A8E
:1004E0008510782A3808FA3A3904031D782A722CC4
:1004F000842A11303902031C842A031D832A953073
:100500003802031C842A722C552A41303A02031CFB
:100510008A2A722CBA0AB908031D922A6530380259
:10052000031C932A4916491CC72A3A08B100B20194
:100530000310B10DB20DB10DB20DB10DB20D3108F8
:10054000A6003208A7004130A800A901DD20BC00A8
:100550008030A100212046305A206F305A2075305B
:100560005A206E305A2064305A2020305A2073307E
:100570005A2069305A20C030212067305A206E300E
:100580005A2061305A206C305A2020305A203C2AA0
:10059000491CE82A012049305A206E305A2069301F
:1005A0005A2074305A2069305A2061305A206C30F9
:1005B0005A2069305A208030A100C03021207A3082
:1005C0005A2065305A202E305A205A205A20462B65
:1005D0000330BC000230A2003C080B20A101C91D61
:1005E000002B3B3040020318F72AC00AFF2AC00143
:1005F000173044020318FE2AC40AFF2AC401042B40
:100600004108C0004508C400051B142BC408031D85
:100610000C2B0C30C600132B0D304402031C132B83
:100620000C304402C600182B4408C60020305A2063
:100630000A30460203181E2B20305A208030A100B9
:10064000460828203A305A200230A40040082920C9
:10065000051B342B0C3044020318312B61305A2017
:10066000332B70305A20342B0130C008031D00306A
:10067000B5001E3040020130031D0030B5040130CA
:1006800086180301B5040319462B4B2C491E492C2F
:10069000F2210130C8000F3048020318532BF22119
:1006A000C80A031D4B2B4911C911F221F221F22175
:1006B000C91C5C2B05145D2B05101230C8001430CA
:1006C00048020318672BF221C80A031D5F2BF22191
:1006D0000730BB00B7214208C100F221491D712B30
:1006E000C9150630BB00B7214208C500F221491DDB
:1006F0007A2BC9150630BB00B7214208BD00033074
:10070000BB00B7214208C7000530BB00B721420833
:10071000BF000830BB00B7214208BE00F221491DCE
:10072000922BC915491C982BC919972B49100120E8
:10073000C919482C8030A10021200230A4003D08B6
:10074000292020305A2001303F02031DAE2B4A30B1
:100750005A2061305A206E305A20262C02303F0237
:10076000031DB92B46305A2065305A2062305A207A
:10077000262C03303F02031DC42B4D305A2061301C
:100780005A2072305A20262C04303F02031DCF2BF2
:1007900041305A2070305A2072305A20262C0530B1
:1007A0003F02031DDA2B4D305A2061305A20793038
:1007B0005A20262C06303F02031DE52B4A305A20D2
:1007C00075305A206E305A20262C07303F02031D08
:1007D000F02B4A305A2075305A206C305A20262C83
:1007E00008303F02031DFB2B41305A2075305A2040
:1007F00067305A20262C09303F02031D062C533047
:100800005A2065305A2070305A20262C0A303F0278
:10081000031D112C4F305A2063305A2074305A2057
:10082000262C0B303F02031D1C2C4E305A206F30FB
:100830005A2076305A20262C0C303F02031D262CDD
:1008400044305A2065305A2063305A20051B3C2C16
:1008500020305A208030A100A4013E08A600A70144
:100860000130D320AA00AB012B20C0302120013061
:10087000A4003E082920482C20305A2027305A2036
:100880008030A100C03021200230A4003E08292081
:100890004A2C722C392A851F522C8316051283127A
:1008A0000512542C8316051683129B30B12001309B
:1008B000C008031D0030B500013086180301B504DF
:1008C0000319632C0515851585140130A900F43032
:1008D000B2200511851185100130A9004A30B220DF
:1008E000C30A492B01204E305A206F305A20203045
:1008F0005A2073305A2069305A2067305A206E309F
:100900005A2061305A208030A100C03021206C3044
:100910005A20203084006030AB20A030840050305A
:10092000AB20203084003030AA20831006188314B6
:100930008318C916831CC91203010618013EC91A7F
:10094000013C031DA92CB60A0319B70A0130B120D6
:100950009C2C0301C91A0130013A0319C912031D65
:10096000C91603010618013EC91A013C031DBE2C1D
:10097000B60A0319B70A0130B120B12C033037028F
:10098000DE30031936020318892C4914392AC72C82
:02400E00503F21
:00000001FF
